:100000008A0115284F295A2982073F3406345B3468
:100010004F3466346D347D3407347F346F34773435
:100020007C3439345E34793471348312031386019D
:10003000850183168601FC01FE018312A001FF30B9
:1000400083160313850080309F00F0014130F100DA
:100050007E08F200F20DF20D720DF83971070318E7
:10006000F00A83129F003C30FB0002208A110A1222
:10007000831203131F15831203131F193B281F102C
:100080001E08F001F9007008FA007908F1007A08FA
:10009000F000F10DF00DF10DF00DF10DF00DF10D81
:1000A000F00DF10DF00DF10DF00DF10DF00DF10D64
:1000B000F00D71080039F10183161E07F1000318D5
:1000C000F00A7108F9007008FA00FD017C087D0251
:1000D000013003180301003C031995287A08F00049
:1000E0007908F100F2010A30F3001030F400F50154
:1000F000F601700DF60DF50D7308F6027208031C7B
:10010000720FF50203188B287308F607720803189C
:10011000720FF5070310F10DF00DF40B792871083B
:10012000F9007008FA00FD0A66287A08F0007908DC
:10013000F100F2010A30F3001030F400F501F6018D
:10014000700DF60DF50D7308F6027208031C720FA0
:10015000F5020318B2287308F60772080318720F25
:10016000F5070310F10DF00DF40BA0287508F00051
:100170007608FF007F08831203138600F0017C08D5
:10018000043E0318F00AF000003C031DC9280614C1
:1001900000297008013C031DD12883120313861423
:1001A00000297008023C031DD92883120313061589
:1001B00000297008033C031DE128831203138615F0
:1001C00000297008043C031DE92883120313061656
:1001D00000297008053C031DF128831203138616BD
:1001E00000297008063C031DF92883120313061723
:1001F00000297008073C031D00298312031386178A
:1002000003307C02013003180301003C03190A2962
:10021000FC0A0B29FC010530F70003208A110A12A1
:10022000FF3083160313850006309F0083120508F4
:100230001039003C03191F290130A0004E298312F8
:100240000313200803194B29F0017E08013E03180F
:10025000F00AF100F2010430F3001030F400F5016F
:10026000F601700DF60DF50D7308F6027208031C09
:10027000720FF502031843297308F6077208031872
:10028000720FF5070310F10DF00DF40B312975080D
:10029000F0007608FE0083120313A0011F28FB0C58
:1002A000FB0C3F30FB050330FB020000FB0B552924
:1002B000000008008E30F800000000000000000080
:1002C00000000000F80B5E290000F70B5A2900001F
:0202D000080024
:00000001FF
